:100000000C9485000C94AD000C94AD000C94AD00E4
:100010000C94AD000C94AD000C94AD000C94AD00AC
:100020000C94AD000C94AD000C94AD000C94AD009C
:100030000C94AD000C94AD000C94AD000C94AD008C
:100040000C94800B0C94AD000C94CD090C94A70972
:100050000C94AD000C94AD000C94AD000C94AD006C
:100060000C94AD000C94AD009F07A207A507A8074C
:10007000AB07AE07B107B407B707BA074E414E4901
:100080004E495459494E46CDCCCC3D0AD7233C1756
:10009000B7D13877CC2B329595E6241FB14F0A00A3
:1000A0000020410000C84200401C4620BCBE4CCA93
:1000B0001B0E5AAEC59D740000000800020100002E
:1000C00003040700000000000000000000000025FD
:1000D0000028002B0000000000240027002A000454
:1000E00004040404040404020202020202030303DF
:1000F00003030301020408102040800102040810D9
:100100002001020408102000000F11241FBECFEFB1
:10011000D8E0DEBFCDBF24E0ACE5B3E001C01D9266
:10012000AC3BB207E1F713E0A0E0B1E0E4EBFFE2A3
:1001300002C005900D92AC35B107D9F710E0C5E8C3
:10014000D0E004C02197FE010E94ED13C438D1070E
:10015000C9F70E94B80C0C94D8170C94000083ECDB
:1001600091E00C94300A4AE050E060E070E00E94B8
:10017000470F97FF03C060E070E0CB0160934C0134
:1001800070934D0180934E0190934F0108954AE082
:1001900050E060E070E00E94470F683E23E0720785
:1001A0008105910524F468EE73E080E090E06093AF
:1001B0003C0170933D0180933E0190933F0108956F
:1001C0000F931F934AE050E060E070E00E94470FF9
:1001D000603127E272078105910524F460E177E23E
:1001E00080E090E00091050410910604209107043E
:1001F00030910804601771078207930744F46093F5
:1002000005047093060480930704909308040091FA
:10021000340110913501209136013091370160177A
:1002200071078207930744F460933401709335019A
:1002300080933601909337016093380170933901B0
:1002400080933A0190933B011F910F910895CF93B2
:10025000DF93EC018AEC91E00E94300ABE01DD0FD1
:10026000880B990B0E94320A86EC91E0DF91CF91C6
:100270000C94300ACF92DF92EF92FF926B017C01D7
:1002800088EC91E00E94300AC701B6010E94320A50
:1002900086EC91E0FF90EF90DF90CF900C94300AC5
:1002A000CF93DF93EC0188EC91E00E94300ABE010D
:1002B000DD0F880B990B0E94320A86EC91E0DF91EA
:1002C000CF910C94300ACF93DF93EC0181309105EC
:1002D00031F460E088E00E94CE0A60E01AC082300B
:1002E000910559F461E088E00E94CE0A60E087E061
:1002F0000E94CE0AC2E0D0E00FC08430910511F414
:1003000060E003C0089771F761E088E00E94CE0AC0
:1003100061E087E00E94CE0ACE01DD0FAA0BBB0B85
:100320008093400190934101A0934201B093430117
:10033000DF91CF9108950F931F934AE050E060E062
:1003400070E00E94470F8B019C01015011092109A7
:100350003109023011052105310578F0643071054D
:100360008105910551F0683071058105910529F0ED
:10037000603171058105910529F4CB011F910F9121
:100380000C9463011F910F91089580910D048823AF
:10039000B9F080914C0190914D01A0914E01B09126
:1003A0004F01181619061A061B0654F40E94740B06
:1003B0006093F4037093F5038093F6039093F7032F
:1003C0000E94740B6093FD037093FE038093FF0300
:1003D000909300040E94740B6093F9037093FA03E6
:1003E0008093FB039093FC0310920D0480913401E1
:1003F00090913501A0913601B091370180930504A9
:1004000090930604A0930704B093080480916001C0
:10041000909161010C941B0B0F931F9380910D041D
:10042000811160C08091480190914901A0914A01D9
:10043000B0914B010097A105B10531F460E084E073
:100440001F910F910C94CE0A81309105A105B10541
:10045000E9F10297A105B10509F044C08091FD03BF
:100460009091FE03A091FF03B0910004892B8A2B89
:100470008B2B21F30E94740B0091FD031091FE035E
:100480002091FF0330910004AB01BC01401B510BD4
:10049000620B730B8091500190915101A091520118
:1004A000B0915301AA27BB2784179507A607B70762
:1004B00068F460E084E00E94CE0A1092FD0310927E
:1004C000FE031092FF03109200040CC061E084E070
:1004D0000E94CE0A80916001909161011F910F915D
:1004E0000C941B0B1F910F9108954AE050E060E0BF
:1004F00070E00E94470F633071058105910550F44B
:10050000609348017093490180934A0190934B0195
:100510000C940C0208952091F0033091F103C9016D
:10052000C4969093F1038093F0033093F3032093E8
:10053000F203813024E09207D0F02091EE03309155
:10054000EF038217930721F41092EF031092EE034A
:100550008091EE039091EF039C012C5C3F4F309310
:10056000F1032093F0039093F3038093F203089533
:100570000F931F93E4E3F1E040E050E0BA01819172
:100580009191A191B191480F591F6A1F7B1F81E082
:10059000E436F807A1F781E000916401109165014C
:1005A0002091660130916701041715072607370768
:1005B00009F080E01F910F9108950F931F93CF933F
:1005C000DF931092F8031092F9031092FA0310923D
:1005D000FB031092FC0381111AC0E4E3F1E0A0E0F8
:1005E000B1E001911191219131914D915D916D9108
:1005F0007D91041715072607370749F421E0E436F3
:10060000F20779F7DF91CF911F910F9108950E9422
:10061000B802882399F08091640190916501A091BE
:100620006601B09167010197A109B1098093640146
:1006300090936501A0936601B09367016DE070E04F
:100640008091F2039091F3030E94A50AE4E3F1E0A4
:10065000C0E0D1E080E090E0DC01419151916191F6
:1006600071914993599369937993840F951FA61FAC
:10067000B71F21E0E436F20781F78093640190937D
:100680006501A0936601B093670180933001909358
:100690003101A0933201B09333010E948B026DE0CF
:1006A00070E08091F2039091F303DF91CF911F915D
:1006B0000F910C94A50ACF93DF93E8E6F1E0C4E331
:1006C000D1E0A0E0B1E041915191619171914993E4
:1006D0005993699379934D935D936D937D9381E0E5
:1006E000EC39F80781F781E0DF91CF910C94DD02BE
:1006F000FF920F931F93CF93DF9300D000D0CDB71D
:10070000DEB704EA13E086E4F82E8EE094E00E945F
:10071000F808892B09F403C58EE094E00E94D608FE
:100720008B3551F41092EB031092EA03D801EF2DB0
:100730001D92EA95E9F7E9CF8D3509F0E1C4E4EAC5
:10074000F3E001900020E9F731978F01045A13403C
:100750001092A3031092A20385E0EDE9F3E0DF011C
:100760001D928A95E9F781E4ECE5F3E0DF011D9243
:100770008A95E9F704301105C4F044E050E064EADA
:1007800073E08DE993E00E9416150430110569F0BD
:10079000A801445051095093A3034093A20368EA6F
:1007A00073E08CE593E00E9416156DE973E08CEC24
:1007B00091E00E940D15892BC9F488EC91E00E940C
:1007C000300A81ED91E00E94300A82EA91E00E94B5
:1007D000300A88ED91E00E94300A8CE991E00E9495
:1007E000300A86EC91E00E94300A99C46DE973E00A
:1007F00083EE91E00E940D15892B49F4609134013C
:1008000070913501809136019091370110C06DE9EA
:1008100073E088EE91E00E940D15892B59F46091E8
:1008200005047091060480910704909108040E94C9
:100830003A0175C46DE973E08DEE91E00E940D15EB
:10084000892B09F057C04AE050E060E070E08CE589
:1008500093E00E94470FAB01BC018091340190915D
:100860003501A0913601B0913701841B950BA60B81
:10087000B70BB7FF07C0B095A095909581959F4F96
:10088000AF4FBF4F00913C0110913D0120913E01BF
:1008900030913F01081719072A073B071CF485E62A
:1008A00090E02BC477FD3BC48091380190913901D1
:1008B000A0913A01B0913B0184179507A607B707AD
:1008C0000CF42DC48091050490910604A0910704B6
:1008D000B0910804481759076A077B0741F0409315
:1008E00005045093060460930704709308040E9463
:1008F000AF0015C46DE973E082EF91E00E940D1521
:10090000892B09F04DC080910D04882319F081E0F6
:1009100090E0BBC280914C0190914D01A0914E019D
:10092000B0914F01181619061A061B06B4F58091EE
:10093000F4039091F503A091F603B091F703892B8E
:100940008A2B8B2B51F10E94740B0091F4031091B0
:10095000F5032091F6033091F703DC01CB01801BF6
:10096000910BA20BB30B00914C0110914D01209102
:100970004E0130914F0180179107A207B3073CF257
:1009800080E090E00E9450011092F4031092F50371
:100990001092F6031092F703C2C380E090E075C294
:1009A0006DE973E087EF91E00E940D15892B09F046
:1009B00048C081E080930D0461E084E00E94CE0A8B
:1009C00080915C0190915D010E941B0B8BE99FE07F
:1009D0000197F1F70E94740B6093090470930A0465
:1009E00080930B0490930C048091440190914501F5
:1009F000A0914601B091470182309105A105B10552
:100A000071F083309105A105B10571F00197A10541
:100A1000B10551F48EE190E0A0E0B0E009C08CE0B7
:100A200090E0A0E0B0E004C081E090E0A0E0B0E0A1
:100A30008093010490930204A0930304B0930404F0
:100A40006EC36DE973E08CEF91E00E940D15892B68
:100A500029F40E94C5010E940C0261C36DE973E094
:100A600081E092E00E940D15892B49F460913801D4
:100A70007091390180913A0190913B01D8CE6DE996
:100A800073E086E092E00E940D15892B29F48CE535
:100A900093E00E94E0004BC16DE973E08BE092E0CF
:100AA0000E940D15892B49F460913C0170913D0124
:100AB00080913E0190913F01BACE6DE973E080E1F3
:100AC00092E00E940D15892B29F48CE593E00E9499
:100AD000C7002DC16DE973E085E192E00E940D151C
:100AE000892B29F48091400190914101CEC16DE99B
:100AF00073E08AE192E00E940D15892B29F48CE5C0
:100B000093E00E949B0113C16DE973E08FE192E0D5
:100B10000E940D15892B29F4809144019091450183
:100B2000B4C16DE973E084E292E00E940D15892B57
:100B3000E9F44AE050E060E070E08CE593E00E9468
:100B4000470F8B019C010150110921093109033024
:100B500011052105310508F0EAC060934401709346
:100B600045018093460190934701E1C06DE973E030
:100B700089E292E00E940D15892B19F40E945B0313
:100B8000B6CE6DE973E08EE292E00E940D15892BDE
:100B900019F40C940000C3C26DE973E083E392E0A2
:100BA0000E940D15892B29F48091480190914901EB
:100BB0006CC16DE973E088E392E00E940D15892B0A
:100BC00029F48CE593E00E947502B1C06DE973E0F1
:100BD0008DE392E00E940D15892B29F480914C0140
:100BE00090914D0152C16DE973E082E492E00E9460
:100BF0000D15892B29F48CE593E00E94B30097C072
:100C00006DE973E087E492E00E940D15892B09F4E9
:100C10008EC06DE973E08CE492E00E940D15892B83
:100C200029F48CE593E00E94020C81C06DE973E029
:100C300081E592E00E940D15892BF1F54AE050E024
:100C400060E070E08CE593E00E94470F97FD12C0D2
:100C5000009138011091390120913A0130913B0106
:100C6000DC01CB01081719072A073B0734F4D90127
:100C7000C80103C080E090E0DC01009134011091D4
:100C800035012091360130913701081719072A07DD
:100C90003B0709F42CCE8093340190933501A09347
:100CA0003601B09337018093050490930604A09316
:100CB0000704B09308043BC06DE973E086E592E059
:100CC0000E940D15892B49F46091500170915101DA
:100CD0008091520190915301AACD6DE973E08BE5AB
:100CE00092E00E940D15892B29F48CE593E00E9477
:100CF000EE0B1DC06DE973E080E692E00E940D15D9
:100D0000892B49F4609154017091550180915601ED
:100D1000909157018CCD6DE973E085E692E00E94D9
:100D20000D15892B41F48CE593E00E94DA0B81E0EC
:100D30008093F803DCCD6DE973E08AE692E00E94CF
:100D40000D15892B01F580915C038532B9F4609112
:100D50005C0170915D0180915E0190915F010E9444
:100D600006129B01AC0160E070E084E393E40E9412
:100D7000F31320E030E040EA52E462C080915C016D
:100D800090915D0182C06DE973E084E792E00E947A
:100D90000D15892B91F5E091A203F091A303E55A7B
:100DA000FC4F8081853229F48CE593E00E94160C7B
:100DB000BECF4AE050E060E070E08CE593E00E9436
:100DC000470F653B71058105910554F46436710543
:100DD000810591054CF464E670E080E090E004C089
:100DE00064EB70E080E090E060935C0170935D01E3
:100DF00080935E0190935F019ACF6DE973E089E77C
:100E000092E00E940D15892B09F042C080915C038D
:100E10008532B9F560916001709161018091620144
:100E2000909163010E9406129B01AC0160E070E0AA
:100E300088E493E40E94F31320E030E040E252E4BF
:100E40000E94601420E030E048EC52E40E946512F9
:100E50000E94D2147F936F938FE692E09F938F93BB
:100E60008E010F5F1F4F1F930F930E942515C8011E
:100E70000E94CA0B0F900F900F900F900F900F9041
:100E80004EC180916001909161010E94500147C163
:100E90006DE973E08EE792E00E940D15892BA1F5B4
:100EA000E091A203F091A303E55AFC4F80818532C3
:100EB00029F48CE593E00E94660C39CF4AE050E0BB
:100EC00060E070E08CE593E00E94470F693C71059B
:100ED0008105910554F4603A7105810591054CF442
:100EE00060EA70E080E090E004C068EC70E080E0D0
:100EF00090E0609360017093610180936201909330
:100F000063010E940C0213CF6DE973E083E892E065
:100F10000E940D15892BC9F568E872E08CE593E015
:100F20000E946A1000E010E0009709F400CF0A3038
:100F3000110510F5F801EC5CFF4F0C94ED130E94C5
:100F40009B011AC00E94750217C00E94020C14C0B7
:100F50000E94E00011C00E94C7000EC00E94B300B2
:100F60000BC00E94EE0B08C00E94DA0B05C00E9465
:100F7000160C02C00E94660C0F5F1F4F68E872E0FB
:100F800080E090E00E946A10CFCF6DE973E08AE8BC
:100F900092E00E940D15892B09F0ADC08FE892E018
:100FA0000E94300A6091F2037091F303072E000C47
:100FB000880B990B0E94320A80EA92E00E941E0A76
:100FC00083EA92E00E94300A609134017091350109
:100FD00080913601909137010E94390F8EEA92E09C
:100FE0000E94300A609148017091490180914A0144
:100FF00090914B010E94390F8BEB92E00E94300AD6
:1010000060913C0170913D0180913E0190913F01C2
:101010000E94390F8AEC92E00E94300A60913801F8
:101020007091390180913A0190913B010E94390FF2
:1010300089ED92E00E94300A60914C0170914D015F
:1010400080914E0190914F010E94390F8CEE92E0F9
:101050000E94300A609140017091410180914201EB
:10106000909143010E94390F88EF92E00E94300A6C
:10107000609158017091590180915A0190915B01E2
:101080000E94390F8CE093E00E94300A6091500179
:101090007091510180915201909153010E94390F3A
:1010A00086E293E00E94300A6091540170915501EC
:1010B00080915601909157010E94390F8EE393E081
:1010C0000E94300A60915C0170915D0180915E0127
:1010D00090915F010E94390F8DE493E00E94300AE5
:1010E0006091600170916101809162019091630152
:1010F0000E94390F14C084E690E00E9427010FC0BF
:101100002091EA033091EB03F901EC55FC4F808309
:101110002F5F3F4F3093EB032093EA03F6CA0F9003
:101120000F900F900F90DF91CF911F910F91FF9033
:101130000895CF92DF92EF92FF920F931F93CF9378
:10114000DF936C017A018B01C0E0D0E0CE15DF05A2
:1011500081F0D8016D918D01D601ED91FC91019046
:10116000F081E02DC6010995892B11F02196EECF73
:101170007E01C701DF91CF911F910F91FF90EF90FA
:10118000DF90CF900895089580E090E00895FC01ED
:10119000538D448D252F30E0842F90E0821B930BDC
:1011A000541710F0CF96089501970895FC01918D82
:1011B000828D981761F0828DDF01A80FB11D5D96B9
:1011C0008C91928D9F5F9F73928F90E008958FEF27
:1011D0009FEF0895FC01918D828D981731F0828DDB
:1011E000E80FF11D858D90E008958FEF9FEF089532
:1011F000FC01918D228D892F90E0805C9F4F821B96
:1012000091098F73992708958EE094E00E94F80861
:1012100021E0892B09F420E0822F0895FC01848DC0
:10122000DF01A80FB11DA35ABF4F2C91848D90E010
:1012300001968F739927848FA689B7892C93A089EB
:10124000B1898C91837080648C93938D848D981375
:1012500006C00288F389E02D80818F7D8083089508
:10126000EF92FF920F931F93CF93DF93EC0181E0F6
:10127000888F9B8D8C8D981305C0E889F9898081B2
:1012800085FD26C0F62E0B8D10E00F5F1F4F0F73EC
:101290001127E02E8C8DE8120CC00FB607FCFACF98
:1012A000E889F989808185FFF5CFCE010E940E097A
:1012B000F1CF8B8DFE01E80FF11DE35AFF4FF08255
:1012C0009FB7F8940B8FEA89FB89808180620AC0FE
:1012D0009FB7F894EE89FF896083E889F989808156
:1012E0008370806480839FBF81E090E0DF91CF9125
:1012F0001F910F91FF90EF900895CF93DF93EC0132
:10130000888D8823C9F0EA89FB89808185FD05C025
:10131000A889B9898C9186FD0FC00FB607FCF5CF5F
:10132000808185FFF2CFA889B9898C9185FFEDCFA7
:10133000CE010E940E09E7CFDF91CF9108950E9460
:10134000040981110C94780308950E9408151F92D6
:101350000F920FB60F9211242F933F934F935F93E9
:101360006F937F938F939F93AF93BF93EF93FF936D
:101370008EE094E00E940E09FF91EF91BF91AF9132
:101380009F918F917F916F915F914F913F912F919D
:101390000F900FBE0F901F9018951F920F920FB6CF
:1013A0000F9211242F938F939F93EF93FF93E091CC
:1013B0001E04F0911F048081E0912404F091250423
:1013C00082FD12C09081809127048F5F8F732091DE
:1013D0002804821751F0E0912704F0E0E25FFB4F10
:1013E000958F8093270401C08081FF91EF919F9199
:1013F0008F912F910F900FBE0F901F90189590E036
:10140000FC01ED50FF4F2491FC01E152FF4F84910C
:10141000882399F090E0880F991FFC01EB52FF4F51
:10142000A591B491FC01E553FF4F859194918FB73D
:10143000F894EC91E22BEC938FBF0895009769F03C
:10144000FC0101900020E9F73197AF01481B590BCF
:10145000BC018EE094E00C94990880E090E008953F
:101460000C941E0A8F929F92AF92BF92CF92DF92FE
:10147000EF92FF920F931F93CF93DF93CDB7DEB719
:10148000A1970FB6F894DEBF0FBECDBF6B017C01F4
:1014900097FF2BC06DE28EE094E00E9430098C0132
:1014A00022273327A9012C193D094E095F0919A2EA
:1014B000CE0181967C019AE0892E912CA12CB12C31
:1014C000CA01B901A50194010E945B13605DF70197
:1014D00062937F01211531054105510589F7CF013F
:1014E0000E941E0A800F911F1DC09B01AC0119A212
:1014F0008E010F5D1F4F8AE0C82ED12CE12CF12CFC
:10150000CA01B901A70196010E945B13605DF80151
:1015100062938F01211531054105510589F7CF01EE
:101520000E941E0AA1960FB6F894DEBF0FBECDBF73
:10153000DF91CF911F910F91FF90EF90DF90CF90AF
:10154000BF90AF909F908F900895CF92DF92EF92CF
:10155000FF920F931F93CF93DF937B01C4E3D1E0FE
:1015600000E010E0845391406C010E151F0560F4FB
:10157000B6016C0F7D1F44E050E0CE010E94331392
:101580000F5F1F4F2496F1CFC701DF91CF911F91BD
:101590000F91FF90EF90DF90CF90089590E0FC01C5
:1015A000E954FF4F2491FC01ED50FF4F3491FC01B1
:1015B000E152FF4FE491EE2309F43CC0222339F1BC
:1015C000233091F038F42130A9F0223001F584B5B0
:1015D0008F7D12C0273091F02830A1F02430B9F46B
:1015E000809180008F7D03C0809180008F778093F1
:1015F00080000DC084B58F7784BD09C08091B00094
:101600008F7703C08091B0008F7D8093B000F0E0B1
:10161000EE0FFF1FE553FF4FA591B4919FB7F894CC
:10162000611104C08C913095382302C0EC913E2B9F
:101630003C939FBF0895CF93DF93EC0186E00E9417
:10164000FF09209711F460E004C0CF3FD10531F4C9
:1016500061E086E0DF91CF910C94CE0AEDEBF0E0F3
:10166000E491E330F9F048F4E130B9F0E230A1F56B
:1016700084B5806284BDC8BD34C0E730E9F0E8308D
:1016800019F1E43049F580918000806280938000F8
:10169000D0938B00C0938A0024C084B5806884BD39
:1016A000C7BD1FC080918000806880938000D09368
:1016B0008900C093880015C08091B0008068809335
:1016C000B000C093B3000DC08091B00080628093E1
:1016D000B000C093B40005C0C038D1050CF0B8CF3D
:1016E000B2CFDF91CF9108952FB7F8946091B404F1
:1016F0007091B5048091B6049091B7042FBF0895FE
:101700001F920F920FB60F9211242F933F938F9336
:101710009F93AF93BF938091B4049091B504A0912F
:10172000B604B091B7043091B30423E0230F2D37F2
:1017300020F40196A11DB11D05C026E8230F0296D5
:10174000A11DB11D2093B3048093B4049093B504FC
:10175000A093B604B093B7048091AF049091B00405
:10176000A091B104B091B2040196A11DB11D809366
:10177000AF049093B004A093B104B093B204BF91AE
:10178000AF919F918F913F912F910F900FBE0F902E
:101790001F901895CF93DF93EC0188EC91E00E94A5
:1017A000300ACE010E94300A86EC91E0DF91CF91A1
:1017B0000C94300A4AE050E060E070E00E94470F6D
:1017C00097FF03C060E070E0CB0160935401709319
:1017D0005501809356019093570108954AE050E0D7
:1017E00060E070E00E94470F97FF03C060E070E088
:1017F000CB016093500170935101809352019093FB
:10180000530108954AE050E060E070E00E94470F05
:10181000623071058105910540F460935801709321
:10182000590180935A0190935B010895EF92FF92C2
:101830000F931F93CF93DF93CDB7DEB70DB71EB7CE
:10184000FC0101900020E9F7AF01481B590B425001
:1018500051092DB73EB7241B350B0FB6F8943EBF88
:101860000FBE2DBF2F5F3F4F7901BC01C9010E9400
:101870001615C7010E945D1020E030E048EC52E4EC
:101880000E94601420E030E040EA52E40E946512B9
:101890009B01AC0160E070E084E393E40E94F313E9
:1018A0000E94D21460935C0170935D0180935E018D
:1018B00090935F010FB6F8941EBF0FBE0DBFDF916E
:1018C000CF911F910F91FF90EF900895EF92FF92AB
:1018D0000F931F93CF93DF93CDB7DEB70DB71EB72E
:1018E000FC0101900020E9F7AF01481B590B425061
:1018F00051092DB73EB7241B350B0FB6F8943EBFE8
:101900000FBE2DBF2F5F3F4F7901BC01C9010E945F
:101910001615C7010E945D1020E030E048EC52E44B
:101920000E94601420E030E040E252E40E94651220
:101930009B01AC0160E070E088E493E40E94F31343
:101940000E94D214609360017093610180936201E0
:10195000909363010E940C020FB6F8941EBF0FBE55
:101960000DBFDF91CF911F910F91FF90EF900895E0
:10197000789484B5826084BD84B5816084BD85B56A
:10198000826085BD85B5816085BD80916E00816076
:1019900080936E001092810080918100826080931C
:1019A000810080918100816080938100809180001E
:1019B0008160809380008091B10084608093B10049
:1019C0008091B00081608093B00080917A00846043
:1019D00080937A0080917A00826080937A0080916F
:1019E0007A00816080937A0080917A008068809389
:1019F0007A001092C100E0911E04F0911F0482E071
:101A00008083E0911A04F0911B041082E0911C0481
:101A1000F0911D048FEC808310922604E091220443
:101A2000F091230486E08083E0912004F09121046A
:101A3000808180618083E0912004F0912104808185
:101A400088608083E0912004F09121048081806887
:101A50008083E0912004F091210480818F7D808338
:101A60002091F0033091F1038091EE039091EF0308
:101A70002817390721F41092EF031092EE0380919A
:101A8000EE039091EF039093F1038093F003E12C28
:101A9000F12C44E3C42E41E0D42E8091AD0490910A
:101AA000AE04E816F9069CF50E948B020091F20341
:101AB0001091F303C4E3D1E004531140B8016C0F5B
:101AC0007D1F44E050E0CE010E942313249621E0C4
:101AD000C836D20799F70091F2031091F303C0E0E2
:101AE000D1E000501140B8016C0F7D1F44E050E080
:101AF000CE010E9423132496CC16DD06A1F70E9486
:101B0000B802811106C08FEFE81AF80AC6CF0E940A
:101B10005B0382E00E94FF0983E00E94FF0988E0E6
:101B20000E94FF0987E00E94FF0986E00E94FF09EA
:101B300084E00E94FF0960E082E00E94CE0A60E03B
:101B400083E00E94CE0A60E089E00E94CE0A8FEF17
:101B500090E00E941B0B80914001909141010E94F6
:101B600063010E940C028091340190913501A09193
:101B70003601B09137018093050490930604A09339
:101B80000704B09308041092F4031092F503109226
:101B9000F6031092F7031092FD031092FE031092C9
:101BA000FF03109200041092F9031092FA031092AE
:101BB000FB031092FC0330E4C32E36E0D32EE12C5D
:101BC000F12CC1E080910D04882309F4B5C00E9476
:101BD000740B0091090410910A0420910B043091B8
:101BE0000C04DC01CB01801B910BA20BB30B8C32DC
:101BF0009140A105B10508F094C040913401509185
:101C00003501609136017091370180910504909102
:101C10000604A0910704B091080484179507A6074D
:101C2000B7072CF561E08091580190915901A0917E
:101C30005A01B0915B01892B8A2B8B2B09F460E050
:101C400082E00E94CE0A61E083E00E94CE0A60E05A
:101C500083E00E94CE0A8091340190913501A091D9
:101C60003601B09137010197A109B1092AC048177F
:101C700059076A077B070CF04FC061E0809158015B
:101C800090915901A0915A01B0915B01892B8A2B47
:101C90008B2B09F060E082E00E94CE0A61E083E0D5
:101CA0000E94CE0A60E083E00E94CE0A8091340157
:101CB00090913501A0913601B09137010196A11D97
:101CC000B11D8093340190933501A0933601B093F8
:101CD00037012091400130914101409142015091E2
:101CE0004301C701B6010E94CE13609101047091B7
:101CF0000204629FC001639F900D729F900D11249A
:101D00008230910508F463CF880F991F880F991FBF
:101D100005970197F1F75BCF0E94C5010E940C0265
:101D200056CF0E94740B6093090470930A04809349
:101D30000B0490930C045BC08090FD039090FE0315
:101D4000A090FF03B090000481149104A104B10499
:101D500019F18091480190914901A0914A01B091F7
:101D60004B010297A105B105B9F40E94740BAB01B8
:101D7000BC01481959096A097B0980915001909169
:101D80005101A0915201B0915301AA27BB2784179A
:101D90009507A607B70770F18090F9039090FA03B2
:101DA000A090FB03B090FC0381149104A104B10442
:101DB000B9F00E94740BAB01BC01481959096A09BA
:101DC0007B098091540190915501A0915601B091E9
:101DD0005701AA27BB2784179507A607B70768F0FE
:101DE0008091F803882319F080E00E94DD020E94B0
:101DF0009F09E8CE0E940C02CFCFC093F803F0CF2A
:101E0000EEE0F4E01382128288EE93E0A0E0B0E00E
:101E100084839583A683B78385EB91E09183808348
:101E200085EC90E09587848784EC90E0978786879F
:101E300080EC90E0918B808B81EC90E0938B828B97
:101E400082EC90E0958B848B86EC90E0978B868B70
:101E5000118E128E138E148E84E690E09093AC0453
:101E60008093AB0483E190E09093AE048093AD0443
:101E70000895CF93DF930E94320AEC0180EA92E04A
:101E80000E941E0A8C0F9D1FDF91CF910895A0E044
:101E9000B0E0EDE4FFE00C9489135C016B017A0182
:101EA0006115710519F0FB0191838083E114F10440
:101EB00029F0C7010297839708F0E5C0E501219654
:101EC000F5011081812F90E00E946110892B11F0A3
:101ED0005E01F4CF1D3229F42196F501118101E054
:101EE00007C01B3221F4E5012296F501118100E0C3
:101EF000E114F10409F1F0E1EF16F10429F43FC017
:101F000010E3E114F10421F128E0E216F10401F1FB
:101F100054F4E2E0EE16F10421F5812C912CA12C71
:101F2000B0E4BB2E3EC0FAE0EF16F10439F020E138
:101F3000E216F104B1F430C0103319F1FAE0EF2EDB
:101F4000F12CACEC8A2E982CA82CACE0BA2E29C02F
:101F500078E0E72EF12C812C912CA12CE0E1BE2E13
:101F600020C060E070E080E090E897010F2C000C4A
:101F7000440B550B0E945B1349015A0112C01033E8
:101F800059F488818F7D883509F0BACF198122965E
:101F9000026080E1E82EF12C812C912CA12C68E0CC
:101FA000B62E40E060E070E0CB0127010F2C000C62
:101FB00066087708FE0150ED352E310E29E0231515
:101FC00070F42FEB210F2A3118F439EC332E06C0B0
:101FD0002FE9210F2A3118F529EA322E310E232D4F
:101FE00030E02E153F05DCF447FD16C08616970637
:101FF000A806B90670F0A30192010E944B13630D6D
:10200000711D811D911D61307105810520E89207C8
:1020100010F04FEF01C041E021961081CBCF202F6F
:102020002170C114D10471F0442329F02197F601E5
:10203000D183C08307C001FF19C02297F601D18365
:10204000C08314C047FF12C0222329F060E070E073
:1020500080E090E804C06FEF7FEF8FEF9FE722E210
:1020600030E03093BB042093BA0409C0222381F0EE
:1020700090958095709561957F4F8F4F9F4F462F1C
:10208000372F282F12C040E030E020E090E00DC054
:1020900097FFF5CF82E290E09093BB048093BA045F
:1020A0006FEF7FEF8FEF9FE7EACF642F732F822FC1
:1020B000CDB7DEB7E1E10C94A513662777270C9422
:1020C000961091110C94E411803219F089508550CA
:1020D000C8F7089548EB54E00E946F100895FA0184
:1020E000A191B081009719F41097E1F0CD01DC01C6
:1020F000CD010D90002011F4C00113C0FB0121910E
:10210000222319F02015D9F7F3CFFB0121912015D7
:1021100019F41E92119606C02223C1F70D900020DB
:10212000A1F7D001FA01A193B0830895A0E0B0E037
:10213000ECE9F0E10C948E13EC016B016115710573
:1021400019F0FB01918380837E01FFEFEF1AFF0AF4
:102150000881802F90E00E946110892B11F0E70127
:10216000F3CF0D3239F47E0182E0E80EF11C0981D3
:1021700011E008C00B3229F47E0192E0E90EF11C57
:10218000098110E0E701219743E050E064E870E046
:10219000CE010E94E711892BC1F4239645E050E05F
:1021A0006FE770E0CE010E94E711892B09F42596B4
:1021B000C114D10419F0F601D183C0831111F6C006
:1021C00060E070E080E89FE7FAC043E050E06CE731
:1021D00070E0CE010E94E711892B59F4C114D1049B
:1021E00009F4E9C0F2E0EF0EF11CF601F182E082A1
:1021F000E2C020E030E0A901C0E0D0E0F70180EDCE
:10220000A82EA00E89E08A1530F1912F9260B92E88
:10221000812F887012FF04C0811124C0219622C032
:1022200081112197A5E0B0E00E947D13DC01CB0174
:10223000880F991FAA1FBB1F9C01AD012A0D311DDC
:10224000411D511D283989E93807480789E1580798
:1022500048F0166006C09EEFA9120AC013FD40C0E8
:102260001860B12E8FEFE81AF80A00811B2DC6CF37
:10227000802F8F7D8534A1F580818D3211F410611E
:1022800006C08B3221F0319661E070E004C081819C
:10229000329662E070E080538A3018F0E61BF70B4C
:1022A0001FC060E070E060389CE079075CF4DB01FF
:1022B000AA0FBB1FAA0FBB1F6A0F7B1F660F771FDA
:1022C000680F711D3196DF0111978C9180538A3010
:1022D00050F314FF03C0719561957109C60FD71FA4
:1022E00011FF08C0C114D10429F0CF010197F601F4
:1022F00091838083CA01B9010E940412212F2370A7
:10230000233019F04B015C0106C04B015C01B7FAA8
:10231000B094B7F8B09420E030E0A901C501B40151
:102320000E94FF11882309F43EC0D7FF06C0D19553
:10233000C195D1090BE910E002C003EB10E0680180
:10234000F8E1CF1AD10890E2E92EF12CCE15DF0585
:1023500074F0F8012591359145915491C501B4016E
:102360000E9465124B015C01CE19DF09EFCF0450CA
:102370001109F594E7940C151D0541F78A2D880F76
:102380008B2D881F8F3F49F020E030E0A901C50167
:10239000B4010E94FF11811106C082E290E0909387
:1023A000BB048093BA04C501B40109C060E070E0C9
:1023B00080E89FEF04C060E070E080EC9FE7CDB75D
:1023C000DEB7ECE00C94AA13992788270895FB0147
:1023D000DC014150504088F08D9181341CF08B35E8
:1023E0000CF4805E659161341CF06B350CF4605E1A
:1023F000861B611171F3990B0895881BFCCF0E9415
:10240000411208F481E00895E89409C097FB3EF476
:1024100090958095709561957F4F8F4F9F4F992331
:10242000A9F0F92F96E9BB279395F69587957795AF
:102430006795B795F111F8CFFAF4BB0F11F460FF6F
:102440001BC06F5F7F4F8F4F9F4F16C0882311F0C7
:1024500096E911C0772321F09EE8872F762F05C0DB
:10246000662371F096E8862F70E060E02AF09A9576
:10247000660F771F881FDAF7880F9695879597F96B
:102480000895990F0008550FAA0BE0E8FEEF161605
:102490001706E807F907C0F012161306E407F50758
:1024A00098F0621B730B840B950B39F40A2661F0CC
:1024B000232B242B252B21F408950A2609F4A1406F
:1024C000A6958FEF811D811D08950E9478120C94AE
:1024D000E9120E94DB1238F00E94E21220F09523EC
:1024E00011F00C94D2120C94D81211240C941D13D8
:1024F0000E94FA1270F3959FC1F3950F50E0551F9B
:10250000629FF001729FBB27F00DB11D639FAA2748
:10251000F00DB11DAA1F649F6627B00DA11D661F97
:10252000829F2227B00DA11D621F739FB00DA11DB8
:10253000621F839FA00D611D221F749F3327A00D72
:10254000611D231F849F600D211D822F762F6A2F0E
:1025500011249F5750409AF0F1F088234AF0EE0F73
:10256000FF1FBB1F661F771F881F91505040A9F7A0
:102570009E3F510580F00C94D2120C941D135F3FC6
:10258000E4F3983ED4F3869577956795B795F795DC
:10259000E7959F5FC1F7FE2B880F911D9695879554
:1025A00097F9089597F99F6780E870E060E00895D3
:1025B0009FEF80EC089500240A941616170618065B
:1025C0000906089500240A94121613061406050637
:1025D0000895092E0394000C11F4882352F0BB0FC8
:1025E00040F4BF2B11F460FF04C06F5F7F4F8F4F2B
:1025F0009F4F089557FD9058440F551F59F05F3F66
:1026000071F04795880F97FB991F61F09F3F79F014
:1026100087950895121613061406551FF2CF469596
:10262000F1DF08C0161617061806991FF1CF869518
:102630007105610508940895E894BB2766277727FC
:10264000CB0197F90895DC01CB01FC01F999FECF8C
:1026500006C0F2BDE1BDF89A319600B40D9241502A
:102660005040B8F70895DC01CB0103C02D910E94C2
:102670003E1341505040D0F70895262FF999FECFD0
:102680001FBA92BD81BD20BD0FB6F894FA9AF99A8F
:102690000FBE01960895DB018F939F930E947D13D7
:1026A000BF91AF91A29F800D911DA39F900DB29FEE
:1026B000900D11240895A1E21A2EAA1BBB1BFD0147
:1026C0000DC0AA1FBB1FEE1FFF1FA217B307E40711
:1026D000F50720F0A21BB30BE40BF50B661F771F69
:1026E000881F991F1A9469F7609570958095909549
:1026F0009B01AC01BD01CF0108950E94BF13A59FAE
:10270000900DB49F900DA49F800D911D11240895EC
:102710002F923F924F925F926F927F928F929F92F1
:10272000AF92BF92CF92DF92EF92FF920F931F93DF
:10273000CF93DF93CDB7DEB7CA1BDB0B0FB6F89490
:10274000DEBF0FBECDBF09942A88398848885F84D0
:102750006E847D848C849B84AA84B984C884DF8041
:10276000EE80FD800C811B81AA81B981CE0FD11D25
:102770000FB6F894DEBF0FBECDBFED010895A29F46
:10278000B001B39FC001A39F700D811D1124911D45
:10279000B29F700D811D1124911D0895052E97FB88
:1027A0001EF400940E94E51357FD07D00E945B13AE
:1027B00007FC03D04EF40C94E513509540953095EA
:1027C00021953F4F4F4F5F4F08959095809570959D
:1027D00061957F4F8F4F9F4F0895EE0FFF1F05901C
:1027E000F491E02D09945058BB27AA270E940B149E
:1027F0000C94E9120E94DB1238F00E94E21220F0E1
:1028000039F49F3F19F426F40C94D8120EF4E09595
:10281000E7FB0C94D212E92F0E94FA1258F3BA1770
:10282000620773078407950720F079F4A6F50C94E6
:102830001C130EF4E0950B2EBA2FA02D0B01B9013D
:1028400090010C01CA01A0011124FF27591B99F026
:10285000593F50F4503E68F11A16F040A22F232F32
:10286000342F4427585FF3CF469537952795A79582
:10287000F0405395C9F77EF41F16BA0B620B730B29
:10288000840BBAF09150A1F0FF0FBB1F661F771F9A
:10289000881FC2F70EC0BA0F621F731F841F48F44F
:1028A000879577956795B795F7959E3F08F0B0CFD8
:1028B0009395880F08F09927EE0F979587950895BF
:1028C0000E9474140C94E9120E94E21258F00E94C3
:1028D000DB1240F029F45F3F29F00C94D212511121
:1028E0000C941D130C94D8120E94FA1268F39923C9
:1028F000B1F3552391F3951B550BBB27AA276217FC
:102900007307840738F09F5F5F4F220F331F441F08
:10291000AA1FA9F335D00E2E3AF0E0E832D091503C
:102920005040E695001CCAF72BD0FE2F29D0660F29
:10293000771F881FBB1F261737074807AB07B0E86C
:1029400009F0BB0B802DBF01FF2793585F4F3AF072
:102950009E3F510578F00C94D2120C941D135F3FEA
:10296000E4F3983ED4F3869577956795B795F795F8
:102970009F5FC9F7880F911D9695879597F90895E0
:10298000E1E0660F771F881FBB1F6217730784077C
:10299000BA0720F0621B730B840BBA0BEE1F88F78B
:1029A000E09508950E94D9146894B1110C941D13F8
:1029B00008950E94021388F09F5798F0B92F992725
:1029C000B751B0F0E1F0660F771F881F991F1AF01A
:1029D000BA95C9F714C0B13091F00E941C13B1E050
:1029E00008950C941C13672F782F8827B85F39F04F
:1029F000B93FCCF3869577956795B395D9F73EF4B3
:102A000090958095709561957F4F8F4F9F4F08955A
:102A100081E090E0F8940C94D817FB01DC018D91D3
:102A2000019080190110D9F3990B0895FB01DC0185
:102A30004150504048F001900D920020C9F701C06C
:102A40001D9241505040E0F70895AEE0B0E0EBE257
:102A5000F5E10C9496130D891E8986E08C831A8308
:102A600009838FEF9FE79E838D83AE01475E5F4FA3
:102A70006F89788DCE0101960E944715EF81F88508
:102A8000E00FF11F10822E96E4E00C94B213ABE03D
:102A9000B0E0EDE4F5E10C9488136C017B018A0150
:102AA000FC0117821682838181FFCCC1CE01019681
:102AB0003C01F6019381F70193FD859193FF81918C
:102AC0007F01882309F4BAC1853239F493FD8591D9
:102AD00093FF81917F01853229F4B60190E00E9435
:102AE0003E17E7CF912C212C312CFFE1F315D8F0C4
:102AF0008B3279F038F4803279F08332A1F4232DCF
:102B000020611DC08D3261F0803369F4232D216076
:102B100016C0832D8260382EE32DE4603E2E2AC03D
:102B2000F32DF8601DC037FC2DC020ED280F2A3092
:102B300040F08E32B9F436FC81C1232D2064322E50
:102B400019C036FE06C08AE0989E200D1124922EF0
:102B500011C0EAE02E9E200D1124222EF32DF062EA
:102B60003F2E08C08C3621F4832D8068382E02C099
:102B7000883641F4F70193FD859193FF81917F01A0
:102B80008111B3CF982F9F7D9554933028F40C5F1B
:102B90001F4F9FE399830DC0833631F0833771F067
:102BA000833509F059C021C0F801808189830E5F07
:102BB0001F4F88248394912C530113C02801F2E005
:102BC0004F0E511CF801A080B18036FE03C0692D64
:102BD00070E002C06FEF7FEFC5010E9433174C0118
:102BE0008201F32DFF773F2E16C0280122E0420E0E
:102BF000511CF801A080B18036FE03C0692D70E041
:102C000002C06FEF7FEFC5010E9428174C01F32D22
:102C1000F0683F2E820133FC1BC0822D90E08816A5
:102C20009906B0F4B60180E290E00E943E172A9423
:102C3000F4CFF50137FC859137FE81915F01B60134
:102C400090E00E943E1721102A9421E0821A9108F8
:102C50008114910471F7E8C0843611F0893641F58A
:102C6000F80137FE07C060817181828193810C5F1A
:102C70001F4F08C060817181072E000C880B990BD3
:102C80000E5F1F4FF32DFF763F2E97FF09C09095E3
:102C90008095709561957F4F8F4F9F4FF0683F2EC5
:102CA0002AE030E0A3010E947A17882E861845C0DA
:102CB000853731F4232D2F7EB22E2AE030E025C057
:102CC000932D997FB92E8F36C1F018F4883579F09D
:102CD000B5C0803719F0883721F0B0C0E92FE06126
:102CE000BE2EB4FE0DC0FB2DF460BF2E09C034FE15
:102CF0000AC0292F2660B22E06C028E030E005C0A9
:102D000020E130E002C020E132E0F801B7FE07C068
:102D100060817181828193810C5F1F4F06C0608149
:102D2000718180E090E00E5F1F4FA3010E947A172F
:102D3000882E8618FB2DFF773F2E36FE0DC0232DE3
:102D40002E7FA22E891458F434FE0BC032FC09C029
:102D5000832D8E7EA82E05C0B82CA32C03C0B82CC2
:102D600001C0B92CA4FE0FC0FE01E80DF11D808149
:102D7000803321F49A2D997EA92E09C0A2FE06C0A7
:102D8000B394B39404C08A2D867809F0B394A3FC5D
:102D900011C0A0FE06C0B21488F4280C922C9B1817
:102DA0000EC0B21460F4B60180E290E00E943E17BB
:102DB000B394F7CFB21418F42B1802C0982C212C1E
:102DC000A4FE10C0B60180E390E00E943E17A2FE70
:102DD00017C0A1FC03C088E790E002C088E590E03E
:102DE000B6010CC08A2D867859F0A1FE02C08BE294
:102DF00001C080E2A7FC8DE2B60190E00E943E1780
:102E0000891438F4B60180E390E00E943E179A944A
:102E1000F7CF8A94F301E80DF11D8081B60190E0AF
:102E20000E943E178110F5CF222009F442CEB60150
:102E300080E290E00E943E172A94F6CFF601868148
:102E4000978102C08FEF9FEF2B96E2E10C94A413C1
:102E5000FC010590615070400110D8F78095909565
:102E60008E0F9F1F0895FC0161507040019001106A
:102E7000D8F7809590958E0F9F1F08950F931F93FD
:102E8000CF93DF93FB01238121FD03C08FEF9FEFE1
:102E90002CC022FF16C046815781248135814217FC
:102EA000530744F4A081B1819D012F5F3F4F3183CF
:102EB00020838C93268137812F5F3F4F3783268372
:102EC00014C08B01EC01FB010084F185E02D099514
:102ED000892BE1F6D80116968D919C911797019652
:102EE00017969C938E931697CE01DF91CF911F91E9
:102EF0000F910895FA01AA27283051F1203181F16C
:102F0000E8946F936E7F6E5F7F4F8F4F9F4FAF4FF1
:102F1000B1E03ED0B4E03CD0670F781F891F9A1F04
:102F2000A11D680F791F8A1F911DA11D6A0F711DB8
:102F3000811D911DA11D20D009F468943F912AE0C4
:102F4000269F11243019305D3193DEF6CF010895AC
:102F5000462F4770405D4193B3E00FD0C9F7F6CFDD
:102F6000462F4F70405D4A3318F0495D31FD4052A5
:102F7000419302D0A9F7EACFB4E0A695979587953B
:102F800077956795BA95C9F700976105710508951A
:102F90009B01AC010A2E06945795479537952795C6
:102FA000BA95C9F7620F731F841F951FA01D08955E
:042FB000F894FFCFC3
:102FB400000000000000000000000000000000000D
:102FC40000000000000000000000000000000000FD
:102FD40000000000000000000000000000000000ED
:102FE4000F270000000000000000000000000000A7
:102FF40000000000000000000000000000000000CD
:1030040000000000000000000000000000000000BC
:10301400000000000F27000050C30000A08601003C
:1030240088130000020000000300000001000000FB
:103034000000000060EA000020BF02000000000061
:103044008C000000B400000000000000312E322E7D
:10305400300044656570536B794461642E41463198
:10306400000000000030099908C7087D09F808D657
:1030740008EA08284F4B2900280021004746524DF2
:1030840000426F6172643D002C2056657273696F53
:103094006E3D0047504F530047545247005354521B
:1030A4004700474D4F5600534D4F560053544F5011
:1030B40000474D585000534D585000474D584D004F
:1030C400534D584D004753545000535354500047E8
:1030D40053504400535350440052534554005242F9
:1030E4004F540047434C4D0053434C4D0047425509
:1030F40046005342554600574550520053524556D8
:103104000053504F5300474944430053494443003C
:103114004749444500534944450047434D5600251B
:103124006425250053434D56004743484400534308
:10313400484400434F4E46007C0044454247004DFE
:10314400656D6F727920616464726573733A2000EF
:103154000D0A00506F736974696F6E3A2000436FF3
:10316400696C73206D6F64653A20004D6178206D41
:103174006F76656D656E743A20004D617820706FCE
:10318400736974696F6E3A2000536574746C6520BA
:10319400627566666572206D733A200053746570BB
:1031A400206D6F64653A2000526576657273652000
:1031B400646972656374696F6E3A200049646C6572
:1031C40020636F696C732074696D656F7574202852
:1031D4006D73293A200049646C6520656570726FCF
:1031E4006D207772697465206D73293A20004D6FE4
:1031F40076652063757272656E743A2000486F6C50
:0C320400642063757272656E743A2000DD
:00000001FF
